:10000000020006020400C2D3C2D47537007538005E
:1000100075390012006B20B505120131802A20B617
:10002000051200F680227590FF75A0FF853134859A
:10003000303553350FE53275F010A4423585F03672
:10004000E53375F010A442361200DB7003D540C3CF
:10005000E5341200A8A2B6B382B5400AE535120015
:10006000A8E5361200A81200D280A87580FF85800E
:100070003085903185A02EA27792E0A27692E1A2FF
:100080007592E2A27492E3A27392E4A27292E5A244
:100090007192E6A27092E7F532E5B0A28792E5F59B
:1000A0003353307F53333F227E081340051200C57F
:1000B00080031200B8DEF322C2B77F0ADFFED2B798
:1000C0007F46DFFE22C2B77F50DFFED2B77F50DF10
:1000D000FE22C2B77FAADFFED2B722C3E53795342E
:1000E000700AE53895357004E539953685343785DD
:1000F0003538853639227590FF75A0FF85322EA2DE
:100100007292E0A27192E2A27092E3A27792E7A2C9
:100110007692E685312EA27292E1A27192E4A270EB
:1001200092E5A27782E792E7A27682E692E6F5343C
:1001300022E531443F64FF8532F043F03F63F0FF36
:1001400045F0605C7590FF75A0FF8531718530705A
:1001500053707F12026C20B6088573348572358027
:100160000685753485743585327185337053703FDB
:1001700012026C20B615E57375F010A4423585F0B7
:1001800036E57275F010A442368056E57575F010AC
:10019000A4423585F036E57475F010A442368041EE
:1001A00020B6201201ECE412020AF550E412020A11
:1001B000F55112022CE412024AF552E412024AF5F9
:1001C0005380061202F612036B855134E55375F025
:1001D00010A44550F53585F036E55275F010A4426F
:1001E00036227E15DEFE227E2BDEFE227F08C290A6
:1001F000D2911201E7741F139290B392911201E70A
:10020000DFF5D290C2911201E722D2907F087C00E4
:10021000C3309004DCFB80131201E220900D120128
:10022000E7A29013DFF81201E7A290227F08C2A78D
:10023000D2A61201E7741F1392A7B392A61201E788
:10024000DFF5D2A7C2A61201E722D2A77F087C0061
:10025000C330A704DCFB80131201E220A70D1201BA
:10026000E7A2A713DFF81201E7A2A722E5701202A6
:10027000A975F064A485F072F573E5711202A925E1
:1002800073F573E43572F57253720F8572058573D9
:100290000475030E7502101202BB7F0C1202E68574
:1002A000017453740F85007522C0E0C4540F75F0BB
:1002B0000AA4F5F0D0E0540F25F022EC8AF0A4F85F
:1002C000A9F0ED8AF0A429F9E5F03400FAEC8BF0FE
:1002D000A429F9E5F03AFAE43400FCED8BF0A42A05
:1002E000FAEC35F0FB22C3EB13FBEA13FAE913F93E
:1002F000E813F8DFF1227CFC7DFF8D908C90008D5F
:1003000090A2928C90920B8D90A2928C90920A8DDA
:1003100090A2928C9092098D90A2928C9092088DCE
:1003200090A2928C9092078D90A2928C9092068DC2
:1003300090A2928C9092058D90A2928C9092048DB6
:1003400090A2928C9092038D90A2928C9092028DAA
:1003500090A2928C9092018D90A2928C9092008D9E
:100360009053210F852051852150227C3F7DFF8DA8
:10037000A08CA0008DA0A2A58CA0920B8DA0A2A500
:100380008CA0920A8DA0A2A58CA092098DA0A2A5F6
:100390008CA092088DA0A2A58CA092078DA0A2A5EA
:1003A0008CA092068DA0A2A58CA092058DA0A2A5DE
:1003B0008CA092048DA0A2A58CA092038DA0A2A5D2
:1003C0008CA092028DA0A2A58CA092018DA0A2A5C6
:1003D0008CA092008DA053210F852053852152229D
:00000001FF
